:1000000010C017C016C015C014C013C012C011C054
:1000100010C00FC00EC00DC00CC00BC00AC009C07C
:1000200008C011241FBECFE5D1E0DEBFCDBF02D096
:100030003AC0E6CFBA9AD398CB9933C0C29A2FE789
:100040008AE196E0215080409040E1F700C0000036
:10005000C2982FE78AE196E0215080409040E1F776
:1000600000C00000C29A2FE78AE196E0215080404C
:100070009040E1F700C00000C2982FE78AE196E0C7
:10008000215080409040E1F700C00000C29A2FE765
:100090008AE196E0215080409040E1F700C00000E6
:0A00A000CBCFC298C9CFF894FFCF70
:00000001FF
